 IlmThread_dll

 Timestamp is 44d97f53 (Tue Aug 08 23:23:15 2006)

 Preferred load address is 10000000

 Start         Length     Name                   Class
 0001:00000000 000048faH .text                   CODE
 0001:00004900 00000373H .text$x                 CODE
 0001:00004c80 00000025H .text$yc                CODE
 0001:00004cb0 00000016H .text$yd                CODE
 0002:00000000 0000018cH .idata$5                DATA
 0002:0000018c 00000004H .CRT$XCA                DATA
 0002:00000190 00000004H .CRT$XCU                DATA
 0002:00000194 00000004H .CRT$XCZ                DATA
 0002:00000198 00000004H .CRT$XIA                DATA
 0002:0000019c 00000004H .CRT$XIAA               DATA
 0002:000001a0 00000004H .CRT$XIZ                DATA
 0002:000001a8 000009b0H .rdata                  DATA
 0002:00000b58 00000578H .rdata$r                DATA
 0002:000010d0 00000070H .rdata$sxdata           DATA
 0002:00001140 00000004H .rtc$IAA                DATA
 0002:00001144 00000008H .rtc$IMZ                DATA
 0002:0000114c 00000004H .rtc$IZZ                DATA
 0002:00001150 00000004H .rtc$TAA                DATA
 0002:00001154 00000008H .rtc$TMZ                DATA
 0002:0000115c 00000004H .rtc$TZZ                DATA
 0002:00001160 000008f4H .xdata$x                DATA
 0002:00001a54 00000050H .idata$2                DATA
 0002:00001aa4 00000014H .idata$3                DATA
 0002:00001ab8 0000018cH .idata$4                DATA
 0002:00001c44 00000becH .idata$6                DATA
 0002:00002830 00000000H .edata                  DATA
 0003:00000000 000002ecH .data                   DATA
 0003:000002f0 0000036cH .bss                    DATA

  Address         Publics by Value              Rva+Base       Lib:Object

 0000:0000001c       ___safe_se_handler_count   0000001c     <absolute>
 0000:00000000       ___ImageBase               10000000     <linker-defined>
 0001:00000000       ??0Mutex@IlmThread@@QAE@XZ 10001000 f   IlmThreadMutexWin32.obj
 0001:00000040       ??1Mutex@IlmThread@@UAE@XZ 10001040 f   IlmThreadMutexWin32.obj
 0001:00000080       ?lock@Mutex@IlmThread@@ABEXXZ 10001080 f   IlmThreadMutexWin32.obj
 0001:000000c0       ?unlock@Mutex@IlmThread@@ABEXXZ 100010c0 f   IlmThreadMutexWin32.obj
 0001:00000100       ??_EMutex@IlmThread@@UAEPAXI@Z 10001100 f i IlmThreadMutexWin32.obj
 0001:00000100       ??_GMutex@IlmThread@@UAEPAXI@Z 10001100 f i IlmThreadMutexWin32.obj
 0001:00000140       ??0WorkerThread@?A0x6db1a767@IlmThread@@QAE@PAUData@ThreadPool@2@@Z 10001140 f   IlmThreadPool.obj
 0001:000001b0       ?run@WorkerThread@?A0x6db1a767@IlmThread@@UAEXXZ 100011b0 f   IlmThreadPool.obj
 0001:00000390       ??0Data@TaskGroup@IlmThread@@QAE@XZ 10001390 f   IlmThreadPool.obj
 0001:000003d0       ??1Data@TaskGroup@IlmThread@@QAE@XZ 100013d0 f   IlmThreadPool.obj
 0001:00000430       ?addTask@Data@TaskGroup@IlmThread@@QAEXXZ 10001430 f   IlmThreadPool.obj
 0001:00000490       ?removeTask@Data@TaskGroup@IlmThread@@QAEXXZ 10001490 f   IlmThreadPool.obj
 0001:000004d0       ??0Data@ThreadPool@IlmThread@@QAE@XZ 100014d0 f   IlmThreadPool.obj
 0001:000005c0       ??1Data@ThreadPool@IlmThread@@QAE@XZ 100015c0 f   IlmThreadPool.obj
 0001:00000750       ?finish@Data@ThreadPool@IlmThread@@QAEXXZ 10001750 f   IlmThreadPool.obj
 0001:000009f0       ?stopped@Data@ThreadPool@IlmThread@@QBE_NXZ 100019f0 f   IlmThreadPool.obj
 0001:00000a90       ?stop@Data@ThreadPool@IlmThread@@QAEXXZ 10001a90 f   IlmThreadPool.obj
 0001:00000b30       ??0Task@IlmThread@@QAE@PAVTaskGroup@1@@Z 10001b30 f   IlmThreadPool.obj
 0001:00000b60       ??1Task@IlmThread@@UAE@XZ  10001b60 f   IlmThreadPool.obj
 0001:00000b80       ?group@Task@IlmThread@@QAEPAVTaskGroup@2@XZ 10001b80 f   IlmThreadPool.obj
 0001:00000ba0       ??0TaskGroup@IlmThread@@QAE@XZ 10001ba0 f   IlmThreadPool.obj
 0001:00000c30       ??1TaskGroup@IlmThread@@QAE@XZ 10001c30 f   IlmThreadPool.obj
 0001:00000ca0       ??0ThreadPool@IlmThread@@QAE@I@Z 10001ca0 f   IlmThreadPool.obj
 0001:00000d50       ??1ThreadPool@IlmThread@@UAE@XZ 10001d50 f   IlmThreadPool.obj
 0001:00000dd0       ?numThreads@ThreadPool@IlmThread@@QBEHXZ 10001dd0 f   IlmThreadPool.obj
 0001:00000e80       ?setNumThreads@ThreadPool@IlmThread@@QAEXH@Z 10001e80 f   IlmThreadPool.obj
 0001:000011a0       ?addTask@ThreadPool@IlmThread@@QAEXPAVTask@2@@Z 100021a0 f   IlmThreadPool.obj
 0001:000013a0       ?globalThreadPool@ThreadPool@IlmThread@@SAAAV12@XZ 100023a0 f   IlmThreadPool.obj
 0001:000013b0       ?addGlobalTask@ThreadPool@IlmThread@@SAXPAVTask@2@@Z 100023b0 f   IlmThreadPool.obj
 0001:000013d0       ??_GWorkerThread@?A0x6db1a767@IlmThread@@UAEPAXI@Z 100023d0 f i IlmThreadPool.obj
 0001:000013d0       ??_EWorkerThread@?A0x6db1a767@IlmThread@@UAEPAXI@Z 100023d0 f i IlmThreadPool.obj
 0001:00001410       ??1Lock@IlmThread@@QAE@XZ  10002410 f i IlmThreadPool.obj
 0001:00001450       ??_ETask@IlmThread@@UAEPAXI@Z 10002450 f i IlmThreadPool.obj
 0001:00001450       ??_GTask@IlmThread@@UAEPAXI@Z 10002450 f i IlmThreadPool.obj
 0001:00001490       ??_GThreadPool@IlmThread@@UAEPAXI@Z 10002490 f i IlmThreadPool.obj
 0001:00001490       ??_EThreadPool@IlmThread@@UAEPAXI@Z 10002490 f i IlmThreadPool.obj
 0001:000014d0       ??_EArgExc@Iex@@UAEPAXI@Z  100024d0 f i IlmThreadPool.obj
 0001:000014d0       ??_GArgExc@Iex@@UAEPAXI@Z  100024d0 f i IlmThreadPool.obj
 0001:00001510       ??1ArgExc@Iex@@UAE@XZ      10002510 f i IlmThreadPool.obj
 0001:00001540       ??0ArgExc@Iex@@QAE@ABV01@@Z 10002540 f i IlmThreadPool.obj
 0001:00001580       ??0?$list@PAVTask@IlmThread@@V?$allocator@PAVTask@IlmThread@@@std@@@std@@QAE@XZ 10002580 f i IlmThreadPool.obj
 0001:000015f0       ??1?$list@PAVTask@IlmThread@@V?$allocator@PAVTask@IlmThread@@@std@@@std@@QAE@XZ 100025f0 f i IlmThreadPool.obj
 0001:00001650       ?front@?$list@PAVTask@IlmThread@@V?$allocator@PAVTask@IlmThread@@@std@@@std@@QAEAAPAVTask@IlmThread@@XZ 10002650 f i IlmThreadPool.obj
 0001:00001710       ?pop_front@?$list@PAVTask@IlmThread@@V?$allocator@PAVTask@IlmThread@@@std@@@std@@QAEXXZ 10002710 f i IlmThreadPool.obj
 0001:000017a0       ?clear@?$list@PAVTask@IlmThread@@V?$allocator@PAVTask@IlmThread@@@std@@@std@@QAEXXZ 100027a0 f i IlmThreadPool.obj
 0001:00001840       ??0?$list@PAVWorkerThread@?A0x6db1a767@IlmThread@@V?$allocator@PAVWorkerThread@?A0x6db1a767@IlmThread@@@std@@@std@@QAE@XZ 10002840 f i IlmThreadPool.obj
 0001:000018b0       ??1?$list@PAVWorkerThread@?A0x6db1a767@IlmThread@@V?$allocator@PAVWorkerThread@?A0x6db1a767@IlmThread@@@std@@@std@@QAE@XZ 100028b0 f i IlmThreadPool.obj
 0001:00001910       ?clear@?$list@PAVWorkerThread@?A0x6db1a767@IlmThread@@V?$allocator@PAVWorkerThread@?A0x6db1a767@IlmThread@@@std@@@std@@QAEXXZ 10002910 f i IlmThreadPool.obj
 0001:000019b0       ??D?$_Iterator@$00@?$list@PAVWorkerThread@?A0x6db1a767@IlmThread@@V?$allocator@PAVWorkerThread@?A0x6db1a767@IlmThread@@@std@@@std@@QBEAAPAVWorkerThread@?A0x6db1a767@IlmThread@@XZ 100029b0 f i IlmThreadPool.obj
 0001:00001a20       ?_Insert@?$list@PAVTask@IlmThread@@V?$allocator@PAVTask@IlmThread@@@std@@@std@@QAEXV?$_Iterator@$00@12@ABQAVTask@IlmThread@@@Z 10002a20 f i IlmThreadPool.obj
 0001:00001a90       ?erase@?$list@PAVTask@IlmThread@@V?$allocator@PAVTask@IlmThread@@@std@@@std@@QAE?AV?$_Iterator@$00@12@V312@@Z 10002a90 f i IlmThreadPool.obj
 0001:00001b80       ?_Buynode@?$list@PAVTask@IlmThread@@V?$allocator@PAVTask@IlmThread@@@std@@@std@@IAEPAU_Node@?$_List_nod@PAVTask@IlmThread@@V?$allocator@PAVTask@IlmThread@@@std@@@2@XZ 10002b80 f i IlmThreadPool.obj
 0001:00001c90       ?_Insert@?$list@PAVWorkerThread@?A0x6db1a767@IlmThread@@V?$allocator@PAVWorkerThread@?A0x6db1a767@IlmThread@@@std@@@std@@QAEXV?$_Iterator@$00@12@ABQAVWorkerThread@?A0x6db1a767@IlmThread@@@Z 10002c90 f i IlmThreadPool.obj
 0001:00001d00       ?_Buynode@?$list@PAVWorkerThread@?A0x6db1a767@IlmThread@@V?$allocator@PAVWorkerThread@?A0x6db1a767@IlmThread@@@std@@@std@@IAEPAU_Node@?$_List_nod@PAVWorkerThread@?A0x6db1a767@IlmThread@@V?$allocator@PAVWorkerThread@?A0x6db1a767@IlmThread@@@std@@@2@XZ 10002d00 f i IlmThreadPool.obj
 0001:00001e10       ??E?$_Const_iterator@$00@?$list@PAVWorkerThread@?A0x6db1a767@IlmThread@@V?$allocator@PAVWorkerThread@?A0x6db1a767@IlmThread@@@std@@@std@@QAEAAV012@XZ 10002e10 f i IlmThreadPool.obj
 0001:00001ea0       ?_Buynode@?$list@PAVTask@IlmThread@@V?$allocator@PAVTask@IlmThread@@@std@@@std@@IAEPAU_Node@?$_List_nod@PAVTask@IlmThread@@V?$allocator@PAVTask@IlmThread@@@std@@@2@PAU342@0ABQAVTask@IlmThread@@@Z 10002ea0 f i IlmThreadPool.obj
 0001:00001fd0       ?_Incsize@?$list@PAVTask@IlmThread@@V?$allocator@PAVTask@IlmThread@@@std@@@std@@IAEXI@Z 10002fd0 f i IlmThreadPool.obj
 0001:000020e0       ?what@logic_error@std@@UBEPBDXZ 100030e0 f i IlmThreadPool.obj
 0001:00002120       ??_Elogic_error@std@@UAEPAXI@Z 10003120 f i IlmThreadPool.obj
 0001:00002120       ??_Glogic_error@std@@UAEPAXI@Z 10003120 f i IlmThreadPool.obj
 0001:00002190       ??1length_error@std@@UAE@XZ 10003190 f i IlmThreadPool.obj
 0001:000021f0       ??_Glength_error@std@@UAEPAXI@Z 100031f0 f i IlmThreadPool.obj
 0001:000021f0       ??_Elength_error@std@@UAEPAXI@Z 100031f0 f i IlmThreadPool.obj
 0001:00002260       ??0logic_error@std@@QAE@ABV01@@Z 10003260 f i IlmThreadPool.obj
 0001:000022f0       ?allocate@?$allocator@U_Node@?$_List_nod@PAVTask@IlmThread@@V?$allocator@PAVTask@IlmThread@@@std@@@std@@@std@@QAEPAU_Node@?$_List_nod@PAVTask@IlmThread@@V?$allocator@PAVTask@IlmThread@@@std@@@2@I@Z 100032f0 f i IlmThreadPool.obj
 0001:00002330       ?_Buynode@?$list@PAVWorkerThread@?A0x6db1a767@IlmThread@@V?$allocator@PAVWorkerThread@?A0x6db1a767@IlmThread@@@std@@@std@@IAEPAU_Node@?$_List_nod@PAVWorkerThread@?A0x6db1a767@IlmThread@@V?$allocator@PAVWorkerThread@?A0x6db1a767@IlmThread@@@std@@@2@PAU342@0ABQAVWorkerThread@?A0x6db1a767@IlmThread@@@Z 10003330 f i IlmThreadPool.obj
 0001:00002460       ?_Incsize@?$list@PAVWorkerThread@?A0x6db1a767@IlmThread@@V?$allocator@PAVWorkerThread@?A0x6db1a767@IlmThread@@@std@@@std@@IAEXI@Z 10003460 f i IlmThreadPool.obj
 0001:00002570       ?allocate@?$allocator@U_Node@?$_List_nod@PAVWorkerThread@?A0x6db1a767@IlmThread@@V?$allocator@PAVWorkerThread@?A0x6db1a767@IlmThread@@@std@@@std@@@std@@QAEPAU_Node@?$_List_nod@PAVWorkerThread@?A0x6db1a767@IlmThread@@V?$allocator@PAVWorkerThread@?A0x6db1a767@IlmThread@@@std@@@2@I@Z 10003570 f i IlmThreadPool.obj
 0001:000025b0       ??0length_error@std@@QAE@ABV01@@Z 100035b0 f i IlmThreadPool.obj
 0001:00002650       ??E?$_Const_iterator@$00@?$list@PAVTask@IlmThread@@V?$allocator@PAVTask@IlmThread@@@std@@@std@@QAEAAV012@XZ 10003650 f i IlmThreadPool.obj
 0001:000026e0       ??$_Allocate@U_Node@?$_List_nod@PAVTask@IlmThread@@V?$allocator@PAVTask@IlmThread@@@std@@@std@@@std@@YAPAU_Node@?$_List_nod@PAVTask@IlmThread@@V?$allocator@PAVTask@IlmThread@@@std@@@0@IPAU120@@Z 100036e0 f i IlmThreadPool.obj
 0001:00002770       ??1bad_alloc@std@@UAE@XZ   10003770 f i IlmThreadPool.obj
 0001:000027b0       ??_Ebad_alloc@std@@UAEPAXI@Z 100037b0 f i IlmThreadPool.obj
 0001:000027b0       ??_Gbad_alloc@std@@UAEPAXI@Z 100037b0 f i IlmThreadPool.obj
 0001:00002810       ??$_Allocate@U_Node@?$_List_nod@PAVWorkerThread@?A0x6db1a767@IlmThread@@V?$allocator@PAVWorkerThread@?A0x6db1a767@IlmThread@@@std@@@std@@@std@@YAPAU_Node@?$_List_nod@PAVWorkerThread@?A0x6db1a767@IlmThread@@V?$allocator@PAVWorkerThread@?A0x6db1a767@IlmThread@@@std@@@0@IPAU120@@Z 10003810 f i IlmThreadPool.obj
 0001:000028a0       ??0bad_alloc@std@@QAE@ABV01@@Z 100038a0 f i IlmThreadPool.obj
 0001:000028f0       ??0LogicExc@Iex@@QAE@AAV?$basic_stringstream@DU?$char_traits@D@std@@V?$allocator@D@2@@std@@@Z 100038f0 f i IlmThreadSemaphoreWin32.obj
 0001:00002910       ??1LogicExc@Iex@@UAE@XZ    10003910 f i IlmThreadSemaphoreWin32.obj
 0001:00002920       ?errorString@?A0x80da50f8@IlmThread@@YA?AV?$basic_string@DU?$char_traits@D@std@@V?$allocator@D@2@@std@@XZ 10003920 f   IlmThreadSemaphoreWin32.obj
 0001:000029c0       ??1Semaphore@IlmThread@@UAE@XZ 100039c0 f   IlmThreadSemaphoreWin32.obj
 0001:000029e0       ??0Semaphore@IlmThread@@QAE@I@Z 100039e0 f   IlmThreadSemaphoreWin32.obj
 0001:00002ad0       ?wait@Semaphore@IlmThread@@QAEXXZ 10003ad0 f   IlmThreadSemaphoreWin32.obj
 0001:00002bb0       ?post@Semaphore@IlmThread@@QAEXXZ 10003bb0 f   IlmThreadSemaphoreWin32.obj
 0001:00002c90       ?value@Semaphore@IlmThread@@QBEHXZ 10003c90 f   IlmThreadSemaphoreWin32.obj
 0001:00002d80       ??Bsentry@?$basic_ostream@DU?$char_traits@D@std@@@std@@QBE_NXZ 10003d80 f i IlmThreadSemaphoreWin32.obj
 0001:00002d90       ??0_Sentry_base@?$basic_ostream@DU?$char_traits@D@std@@@std@@QAE@AAV12@@Z 10003d90 f i IlmThreadSemaphoreWin32.obj
 0001:00002dc0       ??1_Sentry_base@?$basic_ostream@DU?$char_traits@D@std@@@std@@QAE@XZ 10003dc0 f i IlmThreadSemaphoreWin32.obj
 0001:00002de0       ??_ELogicExc@Iex@@UAEPAXI@Z 10003de0 f i IlmThreadSemaphoreWin32.obj
 0001:00002de0       ??_GLogicExc@Iex@@UAEPAXI@Z 10003de0 f i IlmThreadSemaphoreWin32.obj
 0001:00002e00       ??_GSemaphore@IlmThread@@UAEPAXI@Z 10003e00 f i IlmThreadSemaphoreWin32.obj
 0001:00002e00       ??_ESemaphore@IlmThread@@UAEPAXI@Z 10003e00 f i IlmThreadSemaphoreWin32.obj
 0001:00002e30       ??0sentry@?$basic_ostream@DU?$char_traits@D@std@@@std@@QAE@AAV12@@Z 10003e30 f i IlmThreadSemaphoreWin32.obj
 0001:00002ec0       ??1sentry@?$basic_ostream@DU?$char_traits@D@std@@@std@@QAE@XZ 10003ec0 f i IlmThreadSemaphoreWin32.obj
 0001:00002f30       ??$?6U?$char_traits@D@std@@@std@@YAAAV?$basic_ostream@DU?$char_traits@D@std@@@0@AAV10@PBD@Z 10003f30 f i IlmThreadSemaphoreWin32.obj
 0001:000030f0       ??0LogicExc@Iex@@QAE@ABV01@@Z 100040f0 f i IlmThreadSemaphoreWin32.obj
 0001:00003110       ?supportsThreads@IlmThread@@YA_NXZ 10004110 f   IlmThreadWin32.obj
 0001:00003120       ?threadLoop@?A0xe2ae61f0@IlmThread@@YGIPAX@Z 10004120 f   IlmThreadWin32.obj
 0001:00003140       ??0Thread@IlmThread@@QAE@XZ 10004140 f   IlmThreadWin32.obj
 0001:00003150       ??1Thread@IlmThread@@UAE@XZ 10004150 f   IlmThreadWin32.obj
 0001:00003180       ?start@Thread@IlmThread@@QAEXXZ 10004180 f   IlmThreadWin32.obj
 0001:00003210       ??_EThread@IlmThread@@UAEPAXI@Z 10004210 f i IlmThreadWin32.obj
 0001:00003210       ??_GThread@IlmThread@@UAEPAXI@Z 10004210 f i IlmThreadWin32.obj
 0001:00003246       ??0BaseExc@Iex@@QAE@PBD@Z  10004246 f   Iex_dll:Iex_dll.dll
 0001:0000324c       ?what@BaseExc@Iex@@UBEPBDXZ 1000424c f   Iex_dll:Iex_dll.dll
 0001:00003252       ??0BaseExc@Iex@@QAE@ABV01@@Z 10004252 f   Iex_dll:Iex_dll.dll
 0001:00003258       ??1BaseExc@Iex@@UAE@XZ     10004258 f   Iex_dll:Iex_dll.dll
 0001:0000325e       ??0BaseExc@Iex@@QAE@AAV?$basic_stringstream@DU?$char_traits@D@std@@V?$allocator@D@2@@std@@@Z 1000425e f   Iex_dll:Iex_dll.dll
 0001:00003264       ?throwErrnoExc@Iex@@YAXABV?$basic_string@DU?$char_traits@D@std@@V?$allocator@D@2@@std@@@Z 10004264 f   Iex_dll:Iex_dll.dll
 0001:0000326a       _InitializeCriticalSection@4 1000426a f   kernel32:KERNEL32.dll
 0001:00003270       _DeleteCriticalSection@4   10004270 f   kernel32:KERNEL32.dll
 0001:00003276       _EnterCriticalSection@4    10004276 f   kernel32:KERNEL32.dll
 0001:0000327c       _LeaveCriticalSection@4    1000427c f   kernel32:KERNEL32.dll
 0001:00003282       _LocalFree@4               10004282 f   kernel32:KERNEL32.dll
 0001:00003288       _FormatMessageA@28         10004288 f   kernel32:KERNEL32.dll
 0001:0000328e       _GetLastError@0            1000428e f   kernel32:KERNEL32.dll
 0001:00003294       _CloseHandle@4             10004294 f   kernel32:KERNEL32.dll
 0001:0000329a       _CreateSemaphoreA@16       1000429a f   kernel32:KERNEL32.dll
 0001:000032a0       _WaitForSingleObject@8     100042a0 f   kernel32:KERNEL32.dll
 0001:000032a6       _ReleaseSemaphore@12       100042a6 f   kernel32:KERNEL32.dll
 0001:000032ac       ??0?$basic_string@DU?$char_traits@D@std@@V?$allocator@D@2@@std@@QAE@ABV01@@Z 100042ac f   msvcprt:MSVCP80.dll
 0001:000032b2       ??0?$_String_val@DV?$allocator@D@std@@@std@@QAE@ABV01@@Z 100042b2 f   msvcprt:MSVCP80.dll
 0001:000032b8       ??1?$basic_string@DU?$char_traits@D@std@@V?$allocator@D@2@@std@@QAE@XZ 100042b8 f   msvcprt:MSVCP80.dll
 0001:000032be       ??0?$basic_string@DU?$char_traits@D@std@@V?$allocator@D@2@@std@@QAE@PBD@Z 100042be f   msvcprt:MSVCP80.dll
 0001:000032c4       ?c_str@?$basic_string@DU?$char_traits@D@std@@V?$allocator@D@2@@std@@QBEPBDXZ 100042c4 f   msvcprt:MSVCP80.dll
 0001:000032ca       ??4?$basic_string@DU?$char_traits@D@std@@V?$allocator@D@2@@std@@QAEAAV01@PBD@Z 100042ca f   msvcprt:MSVCP80.dll
 0001:000032d0       ??0?$basic_string@DU?$char_traits@D@std@@V?$allocator@D@2@@std@@QAE@XZ 100042d0 f   msvcprt:MSVCP80.dll
 0001:000032d6       ?_Lock@_Mutex@std@@QAEXXZ  100042d6 f   msvcprt:MSVCP80.dll
 0001:000032dc       ?_Unlock@_Mutex@std@@QAEXXZ 100042dc f   msvcprt:MSVCP80.dll
 0001:000032e2       ?flush@?$basic_ostream@DU?$char_traits@D@std@@@std@@QAEAAV12@XZ 100042e2 f   msvcprt:MSVCP80.dll
 0001:000032e8       ?_Osfx@?$basic_ostream@DU?$char_traits@D@std@@@std@@QAEXXZ 100042e8 f   msvcprt:MSVCP80.dll
 0001:000032ee       ?uncaught_exception@std@@YA_NXZ 100042ee f   msvcprt:MSVCP80.dll
 0001:000032f4       ?setstate@?$basic_ios@DU?$char_traits@D@std@@@std@@QAEXH_N@Z 100042f4 f   msvcprt:MSVCP80.dll
 0001:000032fa       ?sputn@?$basic_streambuf@DU?$char_traits@D@std@@@std@@QAEHPBDH@Z 100042fa f   msvcprt:MSVCP80.dll
 0001:00003300       ?sputc@?$basic_streambuf@DU?$char_traits@D@std@@@std@@QAEHD@Z 10004300 f   msvcprt:MSVCP80.dll
 0001:00003306       ??_D?$basic_stringstream@DU?$char_traits@D@std@@V?$allocator@D@2@@std@@QAEXXZ 10004306 f   msvcprt:MSVCP80.dll
 0001:0000330c       ??$?6DU?$char_traits@D@std@@V?$allocator@D@1@@std@@YAAAV?$basic_ostream@DU?$char_traits@D@std@@@0@AAV10@ABV?$basic_string@DU?$char_traits@D@std@@V?$allocator@D@2@@0@@Z 1000430c f   msvcprt:MSVCP80.dll
 0001:00003312       ??0?$basic_stringstream@DU?$char_traits@D@std@@V?$allocator@D@2@@std@@QAE@H@Z 10004312 f   msvcprt:MSVCP80.dll
 0001:00003318       __RTC_CheckEsp             10004318 f   MSVCRT:stack.obj
 0001:0000333b       @_RTC_CheckStackVars@8     1000433b f   MSVCRT:stack.obj
 0001:00003395       @_RTC_AllocaHelper@12      10004395 f   MSVCRT:stack.obj
 0001:000033c2       @_RTC_CheckStackVars2@12   100043c2 f   MSVCRT:stack.obj
 0001:00003475       __RTC_InitBase             10004475 f   MSVCRT:init.obj
 0001:0000349b       __RTC_Shutdown             1000449b f   MSVCRT:init.obj
 0001:000034ad       ??0type_info@@AAE@ABV0@@Z  100044ad f   MSVCRT:ti_inst.obj
 0001:000034b8       ??_Etype_info@@UAEPAXI@Z   100044b8 f i MSVCRT:ti_inst.obj
 0001:00003501       ??4type_info@@AAEAAV0@ABV0@@Z 10004501 f   MSVCRT:ti_inst.obj
 0001:00003506       ??3@YAXPAX@Z               10004506 f   MSVCRT:MSVCR80.dll
 0001:0000350c       ___CxxFrameHandler3        1000450c f   MSVCRT:MSVCR80.dll
 0001:00003512       __invalid_parameter_noinfo 10004512 f   MSVCRT:MSVCR80.dll
 0001:00003518       __purecall                 10004518 f   MSVCRT:MSVCR80.dll
 0001:0000351e       ??2@YAPAXI@Z               1000451e f   MSVCRT:MSVCR80.dll
 0001:00003524       __CxxThrowException@8      10004524 f   MSVCRT:MSVCR80.dll
 0001:0000352a       ??0exception@std@@QAE@ABV01@@Z 1000452a f   MSVCRT:MSVCR80.dll
 0001:00003530       ??1exception@std@@UAE@XZ   10004530 f   MSVCRT:MSVCR80.dll
 0001:00003536       ??0exception@std@@QAE@XZ   10004536 f   MSVCRT:MSVCR80.dll
 0001:0000353c       ??0exception@std@@QAE@ABQBD@Z 1000453c f   MSVCRT:MSVCR80.dll
 0001:00003542       ?what@exception@std@@UBEPBDXZ 10004542 f   MSVCRT:MSVCR80.dll
 0001:00003548       __onexit                   10004548 f   MSVCRT:atonexit.obj
 0001:000035e7       _atexit                    100045e7 f   MSVCRT:atonexit.obj
 0001:000035fa       __endthreadex              100045fa f   MSVCRT:MSVCR80.dll
 0001:00003600       __beginthreadex            10004600 f   MSVCRT:MSVCR80.dll
 0001:00003606       _NtCurrentTeb              10004606 f i MSVCRT:crtdll.obj
 0001:0000365a       __CRT_INIT@12              1000465a f   MSVCRT:crtdll.obj
 0001:0000390f       __DllMainCRTStartup@12     1000490f f   MSVCRT:crtdll.obj
 0001:000039e2       _DebuggerKnownHandle       100049e2 f   MSVCRT:error.obj
 0001:00003bda       ?_RTC_Failure@@YAXPAXH@Z   10004bda f   MSVCRT:error.obj
 0001:00003c12       ?_RTC_StackFailure@@YAXPAXPBD@Z 10004c12 f   MSVCRT:error.obj
 0001:00003d68       ?_RTC_AllocaFailure@@YAXPAXPAU_RTC_ALLOCA_NODE@@H@Z 10004d68 f   MSVCRT:error.obj
 0001:00003e85       __RTC_UninitUse            10004e85 f   MSVCRT:error.obj
 0001:00003f65       __RTC_NumErrors            10004f65 f   MSVCRT:userapi.obj
 0001:00003f69       __RTC_GetErrDesc           10004f69 f   MSVCRT:userapi.obj
 0001:00003f7d       __RTC_SetErrorType         10004f7d f   MSVCRT:userapi.obj
 0001:00003f9a       __RTC_SetErrorFunc         10004f9a f   MSVCRT:userapi.obj
 0001:00003fb1       __RTC_SetErrorFuncW        10004fb1 f   MSVCRT:userapi.obj
 0001:00003fc8       ?_RTC_GetErrorFunc@@YAP6AHHPBDH00ZZPBX@Z 10004fc8 f   MSVCRT:userapi.obj
 0001:00003fce       ?_RTC_GetErrorFuncW@@YAP6AHHPB_WH00ZZPBX@Z 10004fce f   MSVCRT:userapi.obj
 0001:00003fd4       __CRT_RTC_INITW            10004fd4 f   MSVCRT:MSVCR80.dll
 0001:00003fec       ?__ArrayUnwind@@YGXPAXIHP6EX0@Z@Z 10004fec f   MSVCRT:ehvecdtr.obj
 0001:0000404a       ??_M@YGXPAXIHP6EX0@Z@Z     1000504a f   MSVCRT:ehvecdtr.obj
 0001:000040ae       __unlock                   100050ae f   MSVCRT:MSVCR80.dll
 0001:000040b4       __encode_pointer           100050b4 f   MSVCRT:MSVCR80.dll
 0001:000040ba       ___dllonexit               100050ba f   MSVCRT:MSVCR80.dll
 0001:000040c0       __lock                     100050c0 f   MSVCRT:MSVCR80.dll
 0001:000040c6       __decode_pointer           100050c6 f   MSVCRT:MSVCR80.dll
 0001:000040cc       __SEH_prolog4              100050cc f   MSVCRT:sehprolg4.obj
 0001:00004111       __SEH_epilog4              10005111 f   MSVCRT:sehprolg4.obj
 0001:00004125       __except_handler4          10005125 f   MSVCRT:chandler4gs.obj
 0001:00004148       ___clean_type_info_names   10005148 f   MSVCRT:tncleanup.obj
 0001:00004154       __RTC_Initialize           10005154 f   MSVCRT:initsect.obj
 0001:00004178       __RTC_Terminate            10005178 f   MSVCRT:initsect.obj
 0001:0000419c       __malloc_crt               1000519c f   MSVCRT:MSVCR80.dll
 0001:000041a2       __encoded_null             100051a2 f   MSVCRT:MSVCR80.dll
 0001:000041a8       _free                      100051a8 f   MSVCRT:MSVCR80.dll
 0001:000041b0       __ValidateImageBase        100051b0 f   MSVCRT:pesect.obj
 0001:000041e0       __FindPESection            100051e0 f   MSVCRT:pesect.obj
 0001:00004222       __IsNonwritableInCurrentImage 10005222 f   MSVCRT:pesect.obj
 0001:0000428e       __initterm                 1000528e f   MSVCRT:MSVCR80.dll
 0001:00004294       __initterm_e               10005294 f   MSVCRT:MSVCR80.dll
 0001:0000429a       __amsg_exit                1000529a f   MSVCRT:MSVCR80.dll
 0001:000042a0       ___CppXcptFilter           100052a0 f   MSVCRT:MSVCR80.dll
 0001:000042a6       _DllMain@12                100052a6 f   MSVCRT:dllmain.obj
 0001:000042c6       ___security_init_cookie    100052c6 f   MSVCRT:gs_support.obj
 0001:000044b1       ?_RTC_GetSrcLine@@YAHPAEPA_WKPAH1K@Z 100054b1 f   MSVCRT:pdblkup.obj
 0001:00004727       @__security_check_cookie@4 10005727 f   MSVCRT:secchk.obj
 0001:00004736       ?terminate@@YAXXZ          10005736 f   MSVCRT:MSVCR80.dll
 0001:0000473c       ?_type_info_dtor_internal_method@type_info@@QAEXXZ 1000573c f   MSVCRT:MSVCR80.dll
 0001:0000473c       ??1type_info@@UAE@XZ       1000573c f   MSVCRT:MSVCR80.dll
 0001:00004742       __except_handler4_common   10005742 f   MSVCRT:MSVCR80.dll
 0001:00004748       ___clean_type_info_names_internal 10005748 f   MSVCRT:MSVCR80.dll
 0001:0000474e       ___report_gsfailure        1000574e f   MSVCRT:gs_report.obj
 0001:00004852       __crt_debugger_hook        10005852 f   MSVCRT:MSVCR80.dll
 0001:00004858       _InterlockedExchange@8     10005858 f   kernel32:KERNEL32.dll
 0001:0000485e       _Sleep@4                   1000585e f   kernel32:KERNEL32.dll
 0001:00004864       _InterlockedCompareExchange@12 10005864 f   kernel32:KERNEL32.dll
 0001:0000486a       _RaiseException@16         1000586a f   kernel32:KERNEL32.dll
 0001:00004870       _DebugBreak@0              10005870 f   kernel32:KERNEL32.dll
 0001:00004876       _WideCharToMultiByte@32    10005876 f   kernel32:KERNEL32.dll
 0001:0000487c       _IsDebuggerPresent@0       1000587c f   kernel32:KERNEL32.dll
 0001:00004882       _MultiByteToWideChar@24    10005882 f   kernel32:KERNEL32.dll
 0001:00004888       _lstrlenA@4                10005888 f   kernel32:KERNEL32.dll
 0001:0000488e       _GetProcAddress@8          1000588e f   kernel32:KERNEL32.dll
 0001:00004894       _LoadLibraryA@4            10005894 f   kernel32:KERNEL32.dll
 0001:0000489a       _DisableThreadLibraryCalls@4 1000589a f   kernel32:KERNEL32.dll
 0001:000048a0       _QueryPerformanceCounter@4 100058a0 f   kernel32:KERNEL32.dll
 0001:000048a6       _GetTickCount@0            100058a6 f   kernel32:KERNEL32.dll
 0001:000048ac       _GetCurrentThreadId@0      100058ac f   kernel32:KERNEL32.dll
 0001:000048b2       _GetCurrentProcessId@0     100058b2 f   kernel32:KERNEL32.dll
 0001:000048b8       _GetSystemTimeAsFileTime@4 100058b8 f   kernel32:KERNEL32.dll
 0001:000048be       _FreeLibrary@4             100058be f   kernel32:KERNEL32.dll
 0001:000048c4       _HeapFree@12               100058c4 f   kernel32:KERNEL32.dll
 0001:000048ca       _HeapAlloc@12              100058ca f   kernel32:KERNEL32.dll
 0001:000048d0       _GetProcessHeap@0          100058d0 f   kernel32:KERNEL32.dll
 0001:000048d6       _GetModuleFileNameW@12     100058d6 f   kernel32:KERNEL32.dll
 0001:000048dc       _VirtualQuery@12           100058dc f   kernel32:KERNEL32.dll
 0001:000048e2       _TerminateProcess@8        100058e2 f   kernel32:KERNEL32.dll
 0001:000048e8       _GetCurrentProcess@0       100058e8 f   kernel32:KERNEL32.dll
 0001:000048ee       _UnhandledExceptionFilter@4 100058ee f   kernel32:KERNEL32.dll
 0001:000048f4       _SetUnhandledExceptionFilter@4 100058f4 f   kernel32:KERNEL32.dll
 0002:00000000       __imp_?what@BaseExc@Iex@@UBEPBDXZ 10006000     Iex_dll:Iex_dll.dll
 0002:00000004       __imp_??0BaseExc@Iex@@QAE@ABV01@@Z 10006004     Iex_dll:Iex_dll.dll
 0002:00000008       __imp_??1BaseExc@Iex@@UAE@XZ 10006008     Iex_dll:Iex_dll.dll
 0002:0000000c       __imp_??0BaseExc@Iex@@QAE@AAV?$basic_stringstream@DU?$char_traits@D@std@@V?$allocator@D@2@@std@@@Z 1000600c     Iex_dll:Iex_dll.dll
 0002:00000010       __imp_?throwErrnoExc@Iex@@YAXABV?$basic_string@DU?$char_traits@D@std@@V?$allocator@D@2@@std@@@Z 10006010     Iex_dll:Iex_dll.dll
 0002:00000014       __imp_??0BaseExc@Iex@@QAE@PBD@Z 10006014     Iex_dll:Iex_dll.dll
 0002:00000018       \177Iex_dll_NULL_THUNK_DATA 10006018     Iex_dll:Iex_dll.dll
 0002:0000001c       __imp__InitializeCriticalSection@4 1000601c     kernel32:KERNEL32.dll
 0002:00000020       __imp__DeleteCriticalSection@4 10006020     kernel32:KERNEL32.dll
 0002:00000024       __imp__EnterCriticalSection@4 10006024     kernel32:KERNEL32.dll
 0002:00000028       __imp__LeaveCriticalSection@4 10006028     kernel32:KERNEL32.dll
 0002:0000002c       __imp__LocalFree@4         1000602c     kernel32:KERNEL32.dll
 0002:00000030       __imp__FormatMessageA@28   10006030     kernel32:KERNEL32.dll
 0002:00000034       __imp__GetLastError@0      10006034     kernel32:KERNEL32.dll
 0002:00000038       __imp__CloseHandle@4       10006038     kernel32:KERNEL32.dll
 0002:0000003c       __imp__CreateSemaphoreA@16 1000603c     kernel32:KERNEL32.dll
 0002:00000040       __imp__WaitForSingleObject@8 10006040     kernel32:KERNEL32.dll
 0002:00000044       __imp__ReleaseSemaphore@12 10006044     kernel32:KERNEL32.dll
 0002:00000048       __imp__UnhandledExceptionFilter@4 10006048     kernel32:KERNEL32.dll
 0002:0000004c       __imp__GetCurrentProcess@0 1000604c     kernel32:KERNEL32.dll
 0002:00000050       __imp__TerminateProcess@8  10006050     kernel32:KERNEL32.dll
 0002:00000054       __imp__VirtualQuery@12     10006054     kernel32:KERNEL32.dll
 0002:00000058       __imp__GetModuleFileNameW@12 10006058     kernel32:KERNEL32.dll
 0002:0000005c       __imp__GetProcessHeap@0    1000605c     kernel32:KERNEL32.dll
 0002:00000060       __imp__HeapAlloc@12        10006060     kernel32:KERNEL32.dll
 0002:00000064       __imp__HeapFree@12         10006064     kernel32:KERNEL32.dll
 0002:00000068       __imp__FreeLibrary@4       10006068     kernel32:KERNEL32.dll
 0002:0000006c       __imp__GetSystemTimeAsFileTime@4 1000606c     kernel32:KERNEL32.dll
 0002:00000070       __imp__GetCurrentProcessId@0 10006070     kernel32:KERNEL32.dll
 0002:00000074       __imp__GetCurrentThreadId@0 10006074     kernel32:KERNEL32.dll
 0002:00000078       __imp__GetTickCount@0      10006078     kernel32:KERNEL32.dll
 0002:0000007c       __imp__QueryPerformanceCounter@4 1000607c     kernel32:KERNEL32.dll
 0002:00000080       __imp__DisableThreadLibraryCalls@4 10006080     kernel32:KERNEL32.dll
 0002:00000084       __imp__LoadLibraryA@4      10006084     kernel32:KERNEL32.dll
 0002:00000088       __imp__GetProcAddress@8    10006088     kernel32:KERNEL32.dll
 0002:0000008c       __imp__lstrlenA@4          1000608c     kernel32:KERNEL32.dll
 0002:00000090       __imp__MultiByteToWideChar@24 10006090     kernel32:KERNEL32.dll
 0002:00000094       __imp__IsDebuggerPresent@0 10006094     kernel32:KERNEL32.dll
 0002:00000098       __imp__WideCharToMultiByte@32 10006098     kernel32:KERNEL32.dll
 0002:0000009c       __imp__DebugBreak@0        1000609c     kernel32:KERNEL32.dll
 0002:000000a0       __imp__RaiseException@16   100060a0     kernel32:KERNEL32.dll
 0002:000000a4       __imp__InterlockedCompareExchange@12 100060a4     kernel32:KERNEL32.dll
 0002:000000a8       __imp__Sleep@4             100060a8     kernel32:KERNEL32.dll
 0002:000000ac       __imp__InterlockedExchange@8 100060ac     kernel32:KERNEL32.dll
 0002:000000b0       __imp__SetUnhandledExceptionFilter@4 100060b0     kernel32:KERNEL32.dll
 0002:000000b4       \177KERNEL32_NULL_THUNK_DATA 100060b4     kernel32:KERNEL32.dll
 0002:000000b8       __imp_??0?$basic_string@DU?$char_traits@D@std@@V?$allocator@D@2@@std@@QAE@ABV01@@Z 100060b8     msvcprt:MSVCP80.dll
 0002:000000bc       __imp_??1?$basic_string@DU?$char_traits@D@std@@V?$allocator@D@2@@std@@QAE@XZ 100060bc     msvcprt:MSVCP80.dll
 0002:000000c0       __imp_??0?$basic_string@DU?$char_traits@D@std@@V?$allocator@D@2@@std@@QAE@PBD@Z 100060c0     msvcprt:MSVCP80.dll
 0002:000000c4       __imp_?c_str@?$basic_string@DU?$char_traits@D@std@@V?$allocator@D@2@@std@@QBEPBDXZ 100060c4     msvcprt:MSVCP80.dll
 0002:000000c8       __imp_??4?$basic_string@DU?$char_traits@D@std@@V?$allocator@D@2@@std@@QAEAAV01@PBD@Z 100060c8     msvcprt:MSVCP80.dll
 0002:000000cc       __imp_??0?$basic_string@DU?$char_traits@D@std@@V?$allocator@D@2@@std@@QAE@XZ 100060cc     msvcprt:MSVCP80.dll
 0002:000000d0       __imp_?_Lock@_Mutex@std@@QAEXXZ 100060d0     msvcprt:MSVCP80.dll
 0002:000000d4       __imp_?_Unlock@_Mutex@std@@QAEXXZ 100060d4     msvcprt:MSVCP80.dll
 0002:000000d8       __imp_?flush@?$basic_ostream@DU?$char_traits@D@std@@@std@@QAEAAV12@XZ 100060d8     msvcprt:MSVCP80.dll
 0002:000000dc       __imp_?_Osfx@?$basic_ostream@DU?$char_traits@D@std@@@std@@QAEXXZ 100060dc     msvcprt:MSVCP80.dll
 0002:000000e0       __imp_?uncaught_exception@std@@YA_NXZ 100060e0     msvcprt:MSVCP80.dll
 0002:000000e4       __imp_?setstate@?$basic_ios@DU?$char_traits@D@std@@@std@@QAEXH_N@Z 100060e4     msvcprt:MSVCP80.dll
 0002:000000e8       __imp_?sputn@?$basic_streambuf@DU?$char_traits@D@std@@@std@@QAEHPBDH@Z 100060e8     msvcprt:MSVCP80.dll
 0002:000000ec       __imp_?sputc@?$basic_streambuf@DU?$char_traits@D@std@@@std@@QAEHD@Z 100060ec     msvcprt:MSVCP80.dll
 0002:000000f0       __imp_??_D?$basic_stringstream@DU?$char_traits@D@std@@V?$allocator@D@2@@std@@QAEXXZ 100060f0     msvcprt:MSVCP80.dll
 0002:000000f4       __imp_??$?6DU?$char_traits@D@std@@V?$allocator@D@1@@std@@YAAAV?$basic_ostream@DU?$char_traits@D@std@@@0@AAV10@ABV?$basic_string@DU?$char_traits@D@std@@V?$allocator@D@2@@0@@Z 100060f4     msvcprt:MSVCP80.dll
 0002:000000f8       __imp_??0?$basic_stringstream@DU?$char_traits@D@std@@V?$allocator@D@2@@std@@QAE@H@Z 100060f8     msvcprt:MSVCP80.dll
 0002:000000fc       __imp_??0?$_String_val@DV?$allocator@D@std@@@std@@QAE@ABV01@@Z 100060fc     msvcprt:MSVCP80.dll
 0002:00000100       \177MSVCP80_NULL_THUNK_DATA 10006100     msvcprt:MSVCP80.dll
 0002:00000104       __imp____CppXcptFilter     10006104     MSVCRT:MSVCR80.dll
 0002:00000108       __imp_?terminate@@YAXXZ    10006108     MSVCRT:MSVCR80.dll
 0002:0000010c       __imp_?_type_info_dtor_internal_method@type_info@@QAEXXZ 1000610c     MSVCRT:MSVCR80.dll
 0002:00000110       __imp___except_handler4_common 10006110     MSVCRT:MSVCR80.dll
 0002:00000114       __imp____clean_type_info_names_internal 10006114     MSVCRT:MSVCR80.dll
 0002:00000118       __imp___adjust_fdiv        10006118     MSVCRT:MSVCR80.dll
 0002:0000011c       __imp_??0exception@std@@QAE@ABV01@@Z 1000611c     MSVCRT:MSVCR80.dll
 0002:00000120       __imp___CxxThrowException@8 10006120     MSVCRT:MSVCR80.dll
 0002:00000124       __imp_??2@YAPAXI@Z         10006124     MSVCRT:MSVCR80.dll
 0002:00000128       __imp___purecall           10006128     MSVCRT:MSVCR80.dll
 0002:0000012c       __imp___invalid_parameter_noinfo 1000612c     MSVCRT:MSVCR80.dll
 0002:00000130       __imp____CxxFrameHandler3  10006130     MSVCRT:MSVCR80.dll
 0002:00000134       __imp_??3@YAXPAX@Z         10006134     MSVCRT:MSVCR80.dll
 0002:00000138       __imp___amsg_exit          10006138     MSVCRT:MSVCR80.dll
 0002:0000013c       __imp___initterm_e         1000613c     MSVCRT:MSVCR80.dll
 0002:00000140       __imp___initterm           10006140     MSVCRT:MSVCR80.dll
 0002:00000144       __imp__free                10006144     MSVCRT:MSVCR80.dll
 0002:00000148       __imp___encoded_null       10006148     MSVCRT:MSVCR80.dll
 0002:0000014c       __imp___malloc_crt         1000614c     MSVCRT:MSVCR80.dll
 0002:00000150       __imp___decode_pointer     10006150     MSVCRT:MSVCR80.dll
 0002:00000154       __imp___onexit             10006154     MSVCRT:MSVCR80.dll
 0002:00000158       __imp___lock               10006158     MSVCRT:MSVCR80.dll
 0002:0000015c       __imp____dllonexit         1000615c     MSVCRT:MSVCR80.dll
 0002:00000160       __imp___encode_pointer     10006160     MSVCRT:MSVCR80.dll
 0002:00000164       __imp___unlock             10006164     MSVCRT:MSVCR80.dll
 0002:00000168       __imp___CRT_RTC_INITW      10006168     MSVCRT:MSVCR80.dll
 0002:0000016c       __imp___beginthreadex      1000616c     MSVCRT:MSVCR80.dll
 0002:00000170       __imp_??1exception@std@@UAE@XZ 10006170     MSVCRT:MSVCR80.dll
 0002:00000174       __imp_?what@exception@std@@UBEPBDXZ 10006174     MSVCRT:MSVCR80.dll
 0002:00000178       __imp_??0exception@std@@QAE@ABQBD@Z 10006178     MSVCRT:MSVCR80.dll
 0002:0000017c       __imp___crt_debugger_hook  1000617c     MSVCRT:MSVCR80.dll
 0002:00000180       __imp_??0exception@std@@QAE@XZ 10006180     MSVCRT:MSVCR80.dll
 0002:00000184       __imp___endthreadex        10006184     MSVCRT:MSVCR80.dll
 0002:00000188       \177MSVCR80_NULL_THUNK_DATA 10006188     MSVCRT:MSVCR80.dll
 0002:0000018c       ___xc_a                    1000618c     MSVCRT:cinitexe.obj
 0002:00000194       ___xc_z                    10006194     MSVCRT:cinitexe.obj
 0002:00000198       ___xi_a                    10006198     MSVCRT:cinitexe.obj
 0002:000001a0       ___xi_z                    100061a0     MSVCRT:cinitexe.obj
 0002:000001a8       ??_C@_0P@GHFPNOJB@bad?5allocation?$AA@ 100061a8     IlmThreadMutexWin32.obj
 0002:000001b8       ?collate@?$_Locbase@H@std@@2HB 100061b8     IlmThreadMutexWin32.obj
 0002:000001bc       ?ctype@?$_Locbase@H@std@@2HB 100061bc     IlmThreadMutexWin32.obj
 0002:000001c0       ?monetary@?$_Locbase@H@std@@2HB 100061c0     IlmThreadMutexWin32.obj
 0002:000001c4       ?numeric@?$_Locbase@H@std@@2HB 100061c4     IlmThreadMutexWin32.obj
 0002:000001c8       ?time@?$_Locbase@H@std@@2HB 100061c8     IlmThreadMutexWin32.obj
 0002:000001cc       ?messages@?$_Locbase@H@std@@2HB 100061cc     IlmThreadMutexWin32.obj
 0002:000001d0       ?all@?$_Locbase@H@std@@2HB 100061d0     IlmThreadMutexWin32.obj
 0002:000001d4       ?none@?$_Locbase@H@std@@2HB 100061d4     IlmThreadMutexWin32.obj
 0002:000001d8       ?skipws@?$_Iosb@H@std@@2W4_Fmtflags@12@B 100061d8     IlmThreadMutexWin32.obj
 0002:000001dc       ?unitbuf@?$_Iosb@H@std@@2W4_Fmtflags@12@B 100061dc     IlmThreadMutexWin32.obj
 0002:000001e0       ?uppercase@?$_Iosb@H@std@@2W4_Fmtflags@12@B 100061e0     IlmThreadMutexWin32.obj
 0002:000001e4       ?showbase@?$_Iosb@H@std@@2W4_Fmtflags@12@B 100061e4     IlmThreadMutexWin32.obj
 0002:000001e8       ?showpoint@?$_Iosb@H@std@@2W4_Fmtflags@12@B 100061e8     IlmThreadMutexWin32.obj
 0002:000001ec       ?showpos@?$_Iosb@H@std@@2W4_Fmtflags@12@B 100061ec     IlmThreadMutexWin32.obj
 0002:000001f0       ?left@?$_Iosb@H@std@@2W4_Fmtflags@12@B 100061f0     IlmThreadMutexWin32.obj
 0002:000001f4       ?right@?$_Iosb@H@std@@2W4_Fmtflags@12@B 100061f4     IlmThreadMutexWin32.obj
 0002:000001f8       ?internal@?$_Iosb@H@std@@2W4_Fmtflags@12@B 100061f8     IlmThreadMutexWin32.obj
 0002:000001fc       ?dec@?$_Iosb@H@std@@2W4_Fmtflags@12@B 100061fc     IlmThreadMutexWin32.obj
 0002:00000200       ?oct@?$_Iosb@H@std@@2W4_Fmtflags@12@B 10006200     IlmThreadMutexWin32.obj
 0002:00000204       ?hex@?$_Iosb@H@std@@2W4_Fmtflags@12@B 10006204     IlmThreadMutexWin32.obj
 0002:00000208       ?scientific@?$_Iosb@H@std@@2W4_Fmtflags@12@B 10006208     IlmThreadMutexWin32.obj
 0002:0000020c       ?fixed@?$_Iosb@H@std@@2W4_Fmtflags@12@B 1000620c     IlmThreadMutexWin32.obj
 0002:00000210       ?boolalpha@?$_Iosb@H@std@@2W4_Fmtflags@12@B 10006210     IlmThreadMutexWin32.obj
 0002:00000214       ?_Stdio@?$_Iosb@H@std@@2W4_Fmtflags@12@B 10006214     IlmThreadMutexWin32.obj
 0002:00000218       ?adjustfield@?$_Iosb@H@std@@2W4_Fmtflags@12@B 10006218     IlmThreadMutexWin32.obj
 0002:0000021c       ?basefield@?$_Iosb@H@std@@2W4_Fmtflags@12@B 1000621c     IlmThreadMutexWin32.obj
 0002:00000220       ?floatfield@?$_Iosb@H@std@@2W4_Fmtflags@12@B 10006220     IlmThreadMutexWin32.obj
 0002:00000224       ?goodbit@?$_Iosb@H@std@@2W4_Iostate@12@B 10006224     IlmThreadMutexWin32.obj
 0002:00000228       ?eofbit@?$_Iosb@H@std@@2W4_Iostate@12@B 10006228     IlmThreadMutexWin32.obj
 0002:0000022c       ?failbit@?$_Iosb@H@std@@2W4_Iostate@12@B 1000622c     IlmThreadMutexWin32.obj
 0002:00000230       ?badbit@?$_Iosb@H@std@@2W4_Iostate@12@B 10006230     IlmThreadMutexWin32.obj
 0002:00000234       ?_Hardfail@?$_Iosb@H@std@@2W4_Iostate@12@B 10006234     IlmThreadMutexWin32.obj
 0002:00000238       ?in@?$_Iosb@H@std@@2W4_Openmode@12@B 10006238     IlmThreadMutexWin32.obj
 0002:0000023c       ?out@?$_Iosb@H@std@@2W4_Openmode@12@B 1000623c     IlmThreadMutexWin32.obj
 0002:00000240       ?ate@?$_Iosb@H@std@@2W4_Openmode@12@B 10006240     IlmThreadMutexWin32.obj
 0002:00000244       ?app@?$_Iosb@H@std@@2W4_Openmode@12@B 10006244     IlmThreadMutexWin32.obj
 0002:00000248       ?trunc@?$_Iosb@H@std@@2W4_Openmode@12@B 10006248     IlmThreadMutexWin32.obj
 0002:0000024c       ?_Nocreate@?$_Iosb@H@std@@2W4_Openmode@12@B 1000624c     IlmThreadMutexWin32.obj
 0002:00000250       ?_Noreplace@?$_Iosb@H@std@@2W4_Openmode@12@B 10006250     IlmThreadMutexWin32.obj
 0002:00000254       ?binary@?$_Iosb@H@std@@2W4_Openmode@12@B 10006254     IlmThreadMutexWin32.obj
 0002:00000258       ?beg@?$_Iosb@H@std@@2W4_Seekdir@12@B 10006258     IlmThreadMutexWin32.obj
 0002:0000025c       ?cur@?$_Iosb@H@std@@2W4_Seekdir@12@B 1000625c     IlmThreadMutexWin32.obj
 0002:00000260       ?end@?$_Iosb@H@std@@2W4_Seekdir@12@B 10006260     IlmThreadMutexWin32.obj
 0002:00000268       ??_7Mutex@IlmThread@@6B@   10006268     IlmThreadMutexWin32.obj
 0002:00000270       ??_7WorkerThread@?A0x6db1a767@IlmThread@@6B@ 10006270     IlmThreadPool.obj
 0002:0000027c       ??_7Task@IlmThread@@6B@    1000627c     IlmThreadPool.obj
 0002:00000288       ??_7ThreadPool@IlmThread@@6B@ 10006288     IlmThreadPool.obj
 0002:00000290       ??_7ArgExc@Iex@@6B@        10006290     IlmThreadPool.obj
 0002:00000298       ??_C@_0EL@DLLOMFBF@Attempt?5to?5set?5the?5number?5of?5thr@ 10006298     IlmThreadPool.obj
 0002:000002e8       ??_7length_error@std@@6B@  100062e8     IlmThreadPool.obj
 0002:000002f4       ??_7logic_error@std@@6B@   100062f4     IlmThreadPool.obj
 0002:000002fc       ??_C@_0BB@MOGOBHAF@list?$DMT?$DO?5too?5long?$AA@ 100062fc     IlmThreadPool.obj
 0002:00000314       ??_7bad_alloc@std@@6B@     10006314     IlmThreadPool.obj
 0002:00000320       ??_7LogicExc@Iex@@6B@      10006320     IlmThreadSemaphoreWin32.obj
 0002:0000032c       ??_7Semaphore@IlmThread@@6B@ 1000632c     IlmThreadSemaphoreWin32.obj
 0002:00000330       ??_C@_0BN@GNKBEIOC@Could?5not?5create?5semaphore?5?$CI?$AA@ 10006330     IlmThreadSemaphoreWin32.obj
 0002:00000350       ??_C@_02DMCFFCKO@?$CJ?4?$AA@ 10006350     IlmThreadSemaphoreWin32.obj
 0002:00000354       ??_C@_0BO@OKMBNFDM@Could?5not?5wait?5on?5semaphore?5?$CI?$AA@ 10006354     IlmThreadSemaphoreWin32.obj
 0002:00000374       ??_C@_0BO@KDNOPMKO@Could?5not?5post?5on?5semaphore?5?$CI?$AA@ 10006374     IlmThreadSemaphoreWin32.obj
 0002:00000394       ??_C@_0CD@LHHALIDH@Could?5not?5get?5value?5of?5semaphore@ 10006394     IlmThreadSemaphoreWin32.obj
 0002:000003bc       ??_7Thread@IlmThread@@6B@  100063bc     IlmThreadWin32.obj
 0002:000003c4       ??_C@_0BP@EPDMNPGJ@Cannot?5create?5new?5thread?5?$CI?$CFT?$CJ?4?$AA@ 100063c4     IlmThreadWin32.obj
 0002:000003e8       ??_7type_info@@6B@         100063e8     MSVCRT:ti_inst.obj
 0002:000003ec       __pDefaultRawDllMain       100063ec     MSVCRT:crtdll.obj
 0002:000003ec       __pRawDllMain              100063ec     MSVCRT:crtdll.obj
 0002:000003f0       ??_C@_0BO@GNIAFIKK@Unknown?5Runtime?5Check?5Error?6?$AN?$AA@ 100063f0     MSVCRT:error.obj
 0002:00000410       ??_C@_0CM@NGINOKPC@Stack?5memory?5around?5_alloca?5was?5@ 10006410     MSVCRT:error.obj
 0002:0000043c       ??_C@_0DG@HKJMLLLP@A?5local?5variable?5was?5used?5before@ 1000643c     MSVCRT:error.obj
 0002:00000474       ??_C@_0BN@FFOINMNJ@Stack?5memory?5was?5corrupted?6?$AN?$AA@ 10006474     MSVCRT:error.obj
 0002:00000498       ??_C@_0BBN@GPMLNJCF@A?5cast?5to?5a?5smaller?5data?5type?5ha@ 10006498     MSVCRT:error.obj
 0002:000005b8       ??_C@_0NN@NGPKDKPD@The?5value?5of?5ESP?5was?5not?5properl@ 100065b8     MSVCRT:error.obj
 0002:00000718       ??_C@_0CA@IODNCDPG@Run?9Time?5Check?5Failure?5?$CD?$CFd?5?9?5?$CFs?$AA@ 10006718     MSVCRT:error.obj
 0002:00000738       ??_C@_0BE@GNBOBNCK@Unknown?5Module?5Name?$AA@ 10006738     MSVCRT:error.obj
 0002:0000074c       ??_C@_0BB@PFFGGCJP@Unknown?5Filename?$AA@ 1000674c     MSVCRT:error.obj
 0002:00000760       ??_C@_1EA@NFKNIFJP@?$AAR?$AAu?$AAn?$AA?9?$AAT?$AAi?$AAm?$AAe?$AA?5?$AAC?$AAh?$AAe?$AAc?$AAk?$AA?5?$AAF?$AAa?$AAi?$AAl?$AAu?$AAr?$AAe?$AA?5?$AA?$CD?$AA?$CF?$AAd?$AA?5?$AA?9?$AA?5?$AA?$CF?$AAs?$AA?$AA@ 10006760     MSVCRT:error.obj
 0002:000007a0       ??_C@_1GM@OLMCBDMB@?$AAR?$AAu?$AAn?$AAt?$AAi?$AAm?$AAe?$AA?5?$AAC?$AAh?$AAe?$AAc?$AAk?$AA?5?$AAE?$AAr?$AAr?$AAo?$AAr?$AA?4?$AA?6?$AA?$AN?$AA?5?$AAU?$AAn?$AAa?$AAb?$AAl?$AAe?$AA?5?$AAt?$AAo@ 100067a0     MSVCRT:error.obj
 0002:0000080c       ??_C@_0CG@IAFNJNEE@Stack?5corrupted?5near?5unknown?5var@ 1000680c     MSVCRT:error.obj
 0002:00000834       ??_C@_05MKKEDADM@?$CF?42X?5?$AA@ 10006834     MSVCRT:error.obj
 0002:00000840       ??_C@_0EJ@LJKNEOLN@Stack?5area?5around?5_alloca?5memory@ 10006840     MSVCRT:error.obj
 0002:0000088c       ??_C@_08KJEDNCKC@?$CFs?$CFs?$CFs?$CFs?$AA@ 1000688c     MSVCRT:error.obj
 0002:00000898       ??_C@_02LLMPMKNF@?$DO?5?$AA@ 10006898     MSVCRT:error.obj
 0002:0000089c       ??_C@_01EEMJAFIK@?6?$AA@   1000689c     MSVCRT:error.obj
 0002:000008a0       ??_C@_0BC@KIBAILCI@?$CFs?$CFs?$CFp?$CFs?$CFld?$CFs?$CFd?$CFs?$AA@ 100068a0     MSVCRT:error.obj
 0002:000008b8       ??_C@_0EI@CLEPFNGI@Stack?5area?5around?5_alloca?5memory@ 100068b8     MSVCRT:error.obj
 0002:00000900       ??_C@_0N@MHFFIMFG@?6Address?3?50x?$AA@ 10006900     MSVCRT:error.obj
 0002:00000910       ??_C@_07DFDJCKFN@?6Size?3?5?$AA@ 10006910     MSVCRT:error.obj
 0002:00000918       ??_C@_0CK@DKGBICFE@?6Allocation?5number?5within?5this?5f@ 10006918     MSVCRT:error.obj
 0002:00000944       ??_C@_08OMAHNMHJ@?6Data?3?5?$DM?$AA@ 10006944     MSVCRT:error.obj
 0002:00000950       ??_C@_09FOPFMPEJ@wsprintfA?$AA@ 10006950     MSVCRT:error.obj
 0002:0000095c       ??_C@_0L@GMPLCCII@user32?4dll?$AA@ 1000695c     MSVCRT:error.obj
 0002:00000968       ??_C@_0DA@BEGFPCGG@A?5variable?5is?5being?5used?5without@ 10006968     MSVCRT:error.obj
 0002:00000998       ??_C@_0BP@OGBCLIBO@Stack?5around?5_alloca?5corrupted?$AA@ 10006998     MSVCRT:userapi.obj
 0002:000009b8       ??_C@_0CK@CNLNOEPB@Local?5variable?5used?5before?5initi@ 100069b8     MSVCRT:userapi.obj
 0002:000009e4       ??_C@_0BI@CIGMDCBH@Stack?5memory?5corruption?$AA@ 100069e4     MSVCRT:userapi.obj
 0002:000009fc       ??_C@_0CK@FEGOIOPB@Cast?5to?5smaller?5type?5causing?5los@ 100069fc     MSVCRT:userapi.obj
 0002:00000a28       ??_C@_0BJ@HEGAHDFO@Stack?5pointer?5corruption?$AA@ 10006a28     MSVCRT:userapi.obj
 0002:00000a44       ?ProcessDetach@NativeDll@<CrtImplementationDetails>@@0IB 10006a44     MSVCRT:tncleanup.obj
 0002:00000a48       ?ProcessAttach@NativeDll@<CrtImplementationDetails>@@0IB 10006a48     MSVCRT:tncleanup.obj
 0002:00000a4c       ?ThreadAttach@NativeDll@<CrtImplementationDetails>@@0IB 10006a4c     MSVCRT:tncleanup.obj
 0002:00000a50       ?ThreadDetach@NativeDll@<CrtImplementationDetails>@@0IB 10006a50     MSVCRT:tncleanup.obj
 0002:00000a54       ?ProcessVerifier@NativeDll@<CrtImplementationDetails>@@0IB 10006a54     MSVCRT:tncleanup.obj
 0002:00000a58       ??_C@_0M@EKFFODEC@MSPDB80?4DLL?$AA@ 10006a58     MSVCRT:pdblkup.obj
 0002:00000a64       ??_C@_0BF@BMIHBHCA@EnvironmentDirectory?$AA@ 10006a64     MSVCRT:pdblkup.obj
 0002:00000a7c       ??_C@_0CN@EAEOKKOC@SOFTWARE?2Microsoft?2VisualStudio?2@ 10006a7c     MSVCRT:pdblkup.obj
 0002:00000aac       ??_C@_0M@HLOHPNFA@RegCloseKey?$AA@ 10006aac     MSVCRT:pdblkup.obj
 0002:00000ab8       ??_C@_0BB@HHEIPGME@RegQueryValueExA?$AA@ 10006ab8     MSVCRT:pdblkup.obj
 0002:00000acc       ??_C@_0O@DCOGKJGG@RegOpenKeyExA?$AA@ 10006acc     MSVCRT:pdblkup.obj
 0002:00000adc       ??_C@_0N@JJPEKNFO@ADVAPI32?4DLL?$AA@ 10006adc     MSVCRT:pdblkup.obj
 0002:00000aec       ??_C@_01KDCPPGHE@r?$AA@    10006aec     MSVCRT:pdblkup.obj
 0002:00000af0       ??_C@_0BB@KCIACLNC@PDBOpenValidate5?$AA@ 10006af0     MSVCRT:pdblkup.obj
 0002:00000b10       __load_config_used         10006b10     MSVCRT:loadcfg.obj
 0002:00000b58       ??_R4Mutex@IlmThread@@6B@  10006b58     IlmThreadMutexWin32.obj
 0002:00000b6c       ??_R3Mutex@IlmThread@@8    10006b6c     IlmThreadMutexWin32.obj
 0002:00000b7c       ??_R2Mutex@IlmThread@@8    10006b7c     IlmThreadMutexWin32.obj
 0002:00000b84       ??_R1A@?0A@EA@Mutex@IlmThread@@8 10006b84     IlmThreadMutexWin32.obj
 0002:00000ba0       ??_R4WorkerThread@?A0x6db1a767@IlmThread@@6B@ 10006ba0     IlmThreadPool.obj
 0002:00000bb4       ??_R3WorkerThread@?A0x6db1a767@IlmThread@@8 10006bb4     IlmThreadPool.obj
 0002:00000bc4       ??_R2WorkerThread@?A0x6db1a767@IlmThread@@8 10006bc4     IlmThreadPool.obj
 0002:00000bd0       ??_R1A@?0A@EA@WorkerThread@?A0x6db1a767@IlmThread@@8 10006bd0     IlmThreadPool.obj
 0002:00000bec       ??_R1A@?0A@EA@Thread@IlmThread@@8 10006bec     IlmThreadPool.obj
 0002:00000c08       ??_R3Thread@IlmThread@@8   10006c08     IlmThreadPool.obj
 0002:00000c18       ??_R2Thread@IlmThread@@8   10006c18     IlmThreadPool.obj
 0002:00000c20       ??_R4Task@IlmThread@@6B@   10006c20     IlmThreadPool.obj
 0002:00000c34       ??_R3Task@IlmThread@@8     10006c34     IlmThreadPool.obj
 0002:00000c44       ??_R2Task@IlmThread@@8     10006c44     IlmThreadPool.obj
 0002:00000c4c       ??_R1A@?0A@EA@Task@IlmThread@@8 10006c4c     IlmThreadPool.obj
 0002:00000c68       ??_R4ThreadPool@IlmThread@@6B@ 10006c68     IlmThreadPool.obj
 0002:00000c7c       ??_R3ThreadPool@IlmThread@@8 10006c7c     IlmThreadPool.obj
 0002:00000c8c       ??_R2ThreadPool@IlmThread@@8 10006c8c     IlmThreadPool.obj
 0002:00000c94       ??_R1A@?0A@EA@ThreadPool@IlmThread@@8 10006c94     IlmThreadPool.obj
 0002:00000cb0       ??_R4ArgExc@Iex@@6B@       10006cb0     IlmThreadPool.obj
 0002:00000cc4       ??_R3ArgExc@Iex@@8         10006cc4     IlmThreadPool.obj
 0002:00000cd4       ??_R2ArgExc@Iex@@8         10006cd4     IlmThreadPool.obj
 0002:00000cf4       ??_R1A@?0A@EA@ArgExc@Iex@@8 10006cf4     IlmThreadPool.obj
 0002:00000d10       ??_R1A@?0A@EA@BaseExc@Iex@@8 10006d10     IlmThreadPool.obj
 0002:00000d2c       ??_R3BaseExc@Iex@@8        10006d2c     IlmThreadPool.obj
 0002:00000d3c       ??_R2BaseExc@Iex@@8        10006d3c     IlmThreadPool.obj
 0002:00000d58       ??_R1M@?0A@EA@?$basic_string@DU?$char_traits@D@std@@V?$allocator@D@2@@std@@8 10006d58     IlmThreadPool.obj
 0002:00000d74       ??_R3?$basic_string@DU?$char_traits@D@std@@V?$allocator@D@2@@std@@8 10006d74     IlmThreadPool.obj
 0002:00000d84       ??_R2?$basic_string@DU?$char_traits@D@std@@V?$allocator@D@2@@std@@8 10006d84     IlmThreadPool.obj
 0002:00000d98       ??_R1A@?0A@EA@?$basic_string@DU?$char_traits@D@std@@V?$allocator@D@2@@std@@8 10006d98     IlmThreadPool.obj
 0002:00000db4       ??_R1A@?0A@EA@?$_String_val@DV?$allocator@D@std@@@std@@8 10006db4     IlmThreadPool.obj
 0002:00000dd0       ??_R3?$_String_val@DV?$allocator@D@std@@@std@@8 10006dd0     IlmThreadPool.obj
 0002:00000de0       ??_R2?$_String_val@DV?$allocator@D@std@@@std@@8 10006de0     IlmThreadPool.obj
 0002:00000df0       ??_R1A@?0A@EA@_String_base@std@@8 10006df0     IlmThreadPool.obj
 0002:00000e0c       ??_R3_String_base@std@@8   10006e0c     IlmThreadPool.obj
 0002:00000e1c       ??_R2_String_base@std@@8   10006e1c     IlmThreadPool.obj
 0002:00000e28       ??_R1A@?0A@EA@_Container_base@std@@8 10006e28     IlmThreadPool.obj
 0002:00000e44       ??_R3_Container_base@std@@8 10006e44     IlmThreadPool.obj
 0002:00000e54       ??_R2_Container_base@std@@8 10006e54     IlmThreadPool.obj
 0002:00000e5c       ??_R1M@?0A@EA@?$_String_val@DV?$allocator@D@std@@@std@@8 10006e5c     IlmThreadPool.obj
 0002:00000e78       ??_R1M@?0A@EA@_String_base@std@@8 10006e78     IlmThreadPool.obj
 0002:00000e94       ??_R1M@?0A@EA@_Container_base@std@@8 10006e94     IlmThreadPool.obj
 0002:00000eb0       ??_R1A@?0A@EA@exception@std@@8 10006eb0     IlmThreadPool.obj
 0002:00000ecc       ??_R3exception@std@@8      10006ecc     IlmThreadPool.obj
 0002:00000edc       ??_R2exception@std@@8      10006edc     IlmThreadPool.obj
 0002:00000ee4       ??_R4logic_error@std@@6B@  10006ee4     IlmThreadPool.obj
 0002:00000ef8       ??_R3logic_error@std@@8    10006ef8     IlmThreadPool.obj
 0002:00000f08       ??_R2logic_error@std@@8    10006f08     IlmThreadPool.obj
 0002:00000f14       ??_R1A@?0A@EA@logic_error@std@@8 10006f14     IlmThreadPool.obj
 0002:00000f30       ??_R4length_error@std@@6B@ 10006f30     IlmThreadPool.obj
 0002:00000f44       ??_R3length_error@std@@8   10006f44     IlmThreadPool.obj
 0002:00000f54       ??_R2length_error@std@@8   10006f54     IlmThreadPool.obj
 0002:00000f64       ??_R1A@?0A@EA@length_error@std@@8 10006f64     IlmThreadPool.obj
 0002:00000f80       ??_R4bad_alloc@std@@6B@    10006f80     IlmThreadPool.obj
 0002:00000f94       ??_R3bad_alloc@std@@8      10006f94     IlmThreadPool.obj
 0002:00000fa4       ??_R2bad_alloc@std@@8      10006fa4     IlmThreadPool.obj
 0002:00000fb0       ??_R1A@?0A@EA@bad_alloc@std@@8 10006fb0     IlmThreadPool.obj
 0002:00000fcc       ??_R4LogicExc@Iex@@6B@     10006fcc     IlmThreadSemaphoreWin32.obj
 0002:00000fe0       ??_R3LogicExc@Iex@@8       10006fe0     IlmThreadSemaphoreWin32.obj
 0002:00000ff0       ??_R2LogicExc@Iex@@8       10006ff0     IlmThreadSemaphoreWin32.obj
 0002:00001010       ??_R1A@?0A@EA@LogicExc@Iex@@8 10007010     IlmThreadSemaphoreWin32.obj
 0002:0000102c       ??_R4Semaphore@IlmThread@@6B@ 1000702c     IlmThreadSemaphoreWin32.obj
 0002:00001040       ??_R3Semaphore@IlmThread@@8 10007040     IlmThreadSemaphoreWin32.obj
 0002:00001050       ??_R2Semaphore@IlmThread@@8 10007050     IlmThreadSemaphoreWin32.obj
 0002:00001058       ??_R1A@?0A@EA@Semaphore@IlmThread@@8 10007058     IlmThreadSemaphoreWin32.obj
 0002:00001074       ??_R4Thread@IlmThread@@6B@ 10007074     IlmThreadWin32.obj
 0002:00001088       ??_R4type_info@@6B@        10007088     MSVCRT:ti_inst.obj
 0002:0000109c       ??_R3type_info@@8          1000709c     MSVCRT:ti_inst.obj
 0002:000010ac       ??_R2type_info@@8          100070ac     MSVCRT:ti_inst.obj
 0002:000010b4       ??_R1A@?0A@EA@type_info@@8 100070b4     MSVCRT:ti_inst.obj
 0002:000010d0       ___safe_se_handler_table   100070d0     <linker-defined>
 0002:00001140       ___rtc_iaa                 10007140     MSVCRT:initsect.obj
 0002:0000114c       ___rtc_izz                 1000714c     MSVCRT:initsect.obj
 0002:00001150       ___rtc_taa                 10007150     MSVCRT:initsect.obj
 0002:0000115c       ___rtc_tzz                 1000715c     MSVCRT:initsect.obj
 0002:00001398       __TI7?AVArgExc@Iex@@       10007398     IlmThreadPool.obj
 0002:000013a8       __CTA7?AVArgExc@Iex@@      100073a8     IlmThreadPool.obj
 0002:000013c8       __CT??_R0?AVArgExc@Iex@@@8??0ArgExc@Iex@@QAE@ABV01@@Z68 100073c8     IlmThreadPool.obj
 0002:000013e4       __CT??_R0?AVBaseExc@Iex@@@8??0BaseExc@Iex@@QAE@ABV01@@Z68 100073e4     IlmThreadPool.obj
 0002:00001400       __CT??_R0?AV?$basic_string@DU?$char_traits@D@std@@V?$allocator@D@2@@std@@@8??0?$basic_string@DU?$char_traits@D@std@@V?$allocator@D@2@@std@@QAE@ABV01@@Z2812 10007400     IlmThreadPool.obj
 0002:0000141c       __CT??_R0?AV?$_String_val@DV?$allocator@D@std@@@std@@@8??0?$_String_val@DV?$allocator@D@std@@@std@@QAE@ABV01@@Z112 1000741c     IlmThreadPool.obj
 0002:00001438       __CT??_R0?AV_String_base@std@@@8112 10007438     IlmThreadPool.obj
 0002:00001454       __CT??_R0?AU_Container_base@std@@@8112 10007454     IlmThreadPool.obj
 0002:00001470       __CT??_R0?AVexception@std@@@8??0exception@std@@QAE@ABV01@@Z12 10007470     IlmThreadPool.obj
 0002:00001594       __TI3?AVlength_error@std@@ 10007594     IlmThreadPool.obj
 0002:000015d8       __CTA3?AVlength_error@std@@ 100075d8     IlmThreadPool.obj
 0002:000015e8       __CT??_R0?AVlength_error@std@@@8??0length_error@std@@QAE@ABV01@@Z40 100075e8     IlmThreadPool.obj
 0002:00001604       __CT??_R0?AVlogic_error@std@@@8??0logic_error@std@@QAE@ABV01@@Z40 10007604     IlmThreadPool.obj
 0002:00001704       __TI2?AVbad_alloc@std@@    10007704     IlmThreadPool.obj
 0002:00001714       __CTA2?AVbad_alloc@std@@   10007714     IlmThreadPool.obj
 0002:00001720       __CT??_R0?AVbad_alloc@std@@@8??0bad_alloc@std@@QAE@ABV01@@Z12 10007720     IlmThreadPool.obj
 0002:000018f8       __TI7?AVLogicExc@Iex@@     100078f8     IlmThreadSemaphoreWin32.obj
 0002:00001908       __CTA7?AVLogicExc@Iex@@    10007908     IlmThreadSemaphoreWin32.obj
 0002:00001928       __CT??_R0?AVLogicExc@Iex@@@8??0LogicExc@Iex@@QAE@ABV01@@Z68 10007928     IlmThreadSemaphoreWin32.obj
 0002:00001a54       __IMPORT_DESCRIPTOR_Iex_dll 10007a54     Iex_dll:Iex_dll.dll
 0002:00001a68       __IMPORT_DESCRIPTOR_KERNEL32 10007a68     kernel32:KERNEL32.dll
 0002:00001a7c       __IMPORT_DESCRIPTOR_MSVCP80 10007a7c     msvcprt:MSVCP80.dll
 0002:00001a90       __IMPORT_DESCRIPTOR_MSVCR80 10007a90     MSVCRT:MSVCR80.dll
 0002:00001aa4       __NULL_IMPORT_DESCRIPTOR   10007aa4     Iex_dll:Iex_dll.dll
 0003:00000004       ??_R0?AVMutex@IlmThread@@@8 10009004     IlmThreadMutexWin32.obj
 0003:00000028       ??_R0?AVWorkerThread@?A0x6db1a767@IlmThread@@@8 10009028     IlmThreadPool.obj
 0003:0000005c       ??_R0?AVThread@IlmThread@@@8 1000905c     IlmThreadPool.obj
 0003:0000007c       ??_R0?AVTask@IlmThread@@@8 1000907c     IlmThreadPool.obj
 0003:0000009c       ??_R0?AVThreadPool@IlmThread@@@8 1000909c     IlmThreadPool.obj
 0003:000000c0       ??_R0?AVArgExc@Iex@@@8     100090c0     IlmThreadPool.obj
 0003:000000dc       ??_R0?AVBaseExc@Iex@@@8    100090dc     IlmThreadPool.obj
 0003:000000f8       ??_R0?AV?$basic_string@DU?$char_traits@D@std@@V?$allocator@D@2@@std@@@8 100090f8     IlmThreadPool.obj
 0003:00000144       ??_R0?AV?$_String_val@DV?$allocator@D@std@@@std@@@8 10009144     IlmThreadPool.obj
 0003:0000017c       ??_R0?AV_String_base@std@@@8 1000917c     IlmThreadPool.obj
 0003:0000019c       ??_R0?AU_Container_base@std@@@8 1000919c     IlmThreadPool.obj
 0003:000001c0       ??_R0?AVexception@std@@@8  100091c0     IlmThreadPool.obj
 0003:000001dc       ??_R0?AVlogic_error@std@@@8 100091dc     IlmThreadPool.obj
 0003:000001fc       ??_R0?AVlength_error@std@@@8 100091fc     IlmThreadPool.obj
 0003:0000021c       ??_R0?AVbad_alloc@std@@@8  1000921c     IlmThreadPool.obj
 0003:0000023c       ??_R0?AVLogicExc@Iex@@@8   1000923c     IlmThreadSemaphoreWin32.obj
 0003:00000258       ??_R0?AVSemaphore@IlmThread@@@8 10009258     IlmThreadSemaphoreWin32.obj
 0003:00000280       ??_R0?AVtype_info@@@8      10009280     MSVCRT:ti_inst.obj
 0003:00000298       ?_RTC_ErrorLevels@@3PAHA   10009298     MSVCRT:error.obj
 0003:000002d8       ___native_dllmain_reason   100092d8     MSVCRT:natstart.obj
 0003:000002dc       ___native_vcclrit_reason   100092dc     MSVCRT:natstart.obj
 0003:000002e4       ___security_cookie         100092e4     MSVCRT:gs_cookie.obj
 0003:000002e8       ___security_cookie_complement 100092e8     MSVCRT:gs_cookie.obj
 0003:000002f0       ?gThreadPool@IlmThread@@3VThreadPool@1@A 100092f0     IlmThreadPool.obj
 0003:00000300       ?wsprintffp@@3P6AHPADPBDZZA 10009300     MSVCRT:error.obj
 0003:0000030c       ?__type_info_root_node@@3U__type_info_node@@A 1000930c     MSVCRT:tncleanup.obj
 0003:00000644       __adjust_fdiv              10009644     <common>
 0003:00000648       ___native_startup_state    10009648     <common>
 0003:0000064c       ___native_startup_lock     1000964c     <common>
 0003:00000650       ___dyn_tls_init_callback   10009650     <common>
 0003:00000654       ___onexitend               10009654     <common>
 0003:00000658       ___onexitbegin             10009658     <common>

 entry point at        0001:0000390f

 Static symbols

 0001:00001c3f       __catch$?_Buynode@?$list@PAVTask@IlmThread@@V?$allocator@PAVTask@IlmThread@@@std@@@std@@IAEPAU_Node@?$_List_nod@PAVTask@IlmThread@@V?$allocator@PAVTask@IlmThread@@@std@@@2@XZ$0 10002c3f f i IlmThreadPool.obj
 0001:00001dbf       __catch$?_Buynode@?$list@PAVWorkerThread@?A0x6db1a767@IlmThread@@V?$allocator@PAVWorkerThread@?A0x6db1a767@IlmThread@@@std@@@std@@IAEPAU_Node@?$_List_nod@PAVWorkerThread@?A0x6db1a767@IlmThread@@V?$allocator@PAVWorkerThread@?A0x6db1a767@IlmThread@@@std@@@2@XZ$0 10002dbf f i IlmThreadPool.obj
 0001:00001f88       __catch$?_Buynode@?$list@PAVTask@IlmThread@@V?$allocator@PAVTask@IlmThread@@@std@@@std@@IAEPAU_Node@?$_List_nod@PAVTask@IlmThread@@V?$allocator@PAVTask@IlmThread@@@std@@@2@PAU342@0ABQAVTask@IlmThread@@@Z$0 10002f88 f i IlmThreadPool.obj
 0001:00002418       __catch$?_Buynode@?$list@PAVWorkerThread@?A0x6db1a767@IlmThread@@V?$allocator@PAVWorkerThread@?A0x6db1a767@IlmThread@@@std@@@std@@IAEPAU_Node@?$_List_nod@PAVWorkerThread@?A0x6db1a767@IlmThread@@V?$allocator@PAVWorkerThread@?A0x6db1a767@IlmThread@@@std@@@2@PAU342@0ABQAVWorkerThread@?A0x6db1a767@IlmThread@@@Z$0 10003418 f i IlmThreadPool.obj
 0001:000030c5       __catch$??$?6U?$char_traits@D@std@@@std@@YAAAV?$basic_ostream@DU?$char_traits@D@std@@@0@AAV10@PBD@Z$0 100040c5 f i IlmThreadSemaphoreWin32.obj
 0001:0000360d       _pre_c_init                1000460d f   MSVCRT:crtdll.obj
 0001:000037f9       ___DllMainCRTStartup       100047f9 f   MSVCRT:crtdll.obj
 0001:00003930       ?DebuggerProbe@@YAHK@Z     10004930 f   MSVCRT:error.obj
 0001:00003980       ?DebuggerRuntime@@YAHKHPAXPB_W@Z 10004980 f   MSVCRT:error.obj
 0001:000039ec       ?failwithmessage@@YAXPAXHHPBD@Z 100049ec f   MSVCRT:error.obj
 0001:00003d03       ?_getMemBlockDataString@@YAXPAD00I@Z 10004d03 f   MSVCRT:error.obj
 0001:00003fda       ?ArrayUnwindFilter@@YAHPAU_EXCEPTION_POINTERS@@@Z 10004fda f   MSVCRT:ehvecdtr.obj
 0001:0000435a       ?GetPdbDll@@YAPAUHINSTANCE__@@XZ 1000535a f   MSVCRT:pdblkup.obj
 0001:00004900       __unwindfunclet$??0WorkerThread@?A0x6db1a767@IlmThread@@QAE@PAUData@ThreadPool@2@@Z$0 10005900 f   IlmThreadPool.obj
 0001:00004908       __ehhandler$??0WorkerThread@?A0x6db1a767@IlmThread@@QAE@PAUData@ThreadPool@2@@Z 10005908 f   IlmThreadPool.obj
 0001:00004912       __unwindfunclet$?run@WorkerThread@?A0x6db1a767@IlmThread@@UAEXXZ$0 10005912 f   IlmThreadPool.obj
 0001:0000491a       __ehhandler$?run@WorkerThread@?A0x6db1a767@IlmThread@@UAEXXZ 1000591a f   IlmThreadPool.obj
 0001:00004924       __unwindfunclet$??1Data@TaskGroup@IlmThread@@QAE@XZ$0 10005924 f   IlmThreadPool.obj
 0001:0000492c       __ehhandler$??1Data@TaskGroup@IlmThread@@QAE@XZ 1000592c f   IlmThreadPool.obj
 0001:00004936       __unwindfunclet$??0Data@ThreadPool@IlmThread@@QAE@XZ$0 10005936 f   IlmThreadPool.obj
 0001:0000493e       __unwindfunclet$??0Data@ThreadPool@IlmThread@@QAE@XZ$1 1000593e f   IlmThreadPool.obj
 0001:00004949       __unwindfunclet$??0Data@ThreadPool@IlmThread@@QAE@XZ$2 10005949 f   IlmThreadPool.obj
 0001:00004954       __unwindfunclet$??0Data@ThreadPool@IlmThread@@QAE@XZ$3 10005954 f   IlmThreadPool.obj
 0001:0000495f       __unwindfunclet$??0Data@ThreadPool@IlmThread@@QAE@XZ$4 1000595f f   IlmThreadPool.obj
 0001:0000496a       __unwindfunclet$??0Data@ThreadPool@IlmThread@@QAE@XZ$5 1000596a f   IlmThreadPool.obj
 0001:00004975       __ehhandler$??0Data@ThreadPool@IlmThread@@QAE@XZ 10005975 f   IlmThreadPool.obj
 0001:0000497f       __unwindfunclet$??1Data@ThreadPool@IlmThread@@QAE@XZ$0 1000597f f   IlmThreadPool.obj
 0001:00004987       __unwindfunclet$??1Data@ThreadPool@IlmThread@@QAE@XZ$1 10005987 f   IlmThreadPool.obj
 0001:00004992       __unwindfunclet$??1Data@ThreadPool@IlmThread@@QAE@XZ$2 10005992 f   IlmThreadPool.obj
 0001:0000499d       __unwindfunclet$??1Data@ThreadPool@IlmThread@@QAE@XZ$3 1000599d f   IlmThreadPool.obj
 0001:000049a8       __unwindfunclet$??1Data@ThreadPool@IlmThread@@QAE@XZ$4 100059a8 f   IlmThreadPool.obj
 0001:000049b3       __unwindfunclet$??1Data@ThreadPool@IlmThread@@QAE@XZ$5 100059b3 f   IlmThreadPool.obj
 0001:000049be       __unwindfunclet$??1Data@ThreadPool@IlmThread@@QAE@XZ$6 100059be f   IlmThreadPool.obj
 0001:000049c9       __unwindfunclet$??1Data@ThreadPool@IlmThread@@QAE@XZ$7 100059c9 f   IlmThreadPool.obj
 0001:000049d1       __ehhandler$??1Data@ThreadPool@IlmThread@@QAE@XZ 100059d1 f   IlmThreadPool.obj
 0001:000049db       __unwindfunclet$?finish@Data@ThreadPool@IlmThread@@QAEXXZ$0 100059db f   IlmThreadPool.obj
 0001:000049e3       __unwindfunclet$?finish@Data@ThreadPool@IlmThread@@QAEXXZ$1 100059e3 f   IlmThreadPool.obj
 0001:000049eb       __ehhandler$?finish@Data@ThreadPool@IlmThread@@QAEXXZ 100059eb f   IlmThreadPool.obj
 0001:000049f5       __unwindfunclet$??0TaskGroup@IlmThread@@QAE@XZ$0 100059f5 f   IlmThreadPool.obj
 0001:00004a00       __ehhandler$??0TaskGroup@IlmThread@@QAE@XZ 10005a00 f   IlmThreadPool.obj
 0001:00004a0a       __unwindfunclet$??0ThreadPool@IlmThread@@QAE@I@Z$0 10005a0a f   IlmThreadPool.obj
 0001:00004a15       __ehhandler$??0ThreadPool@IlmThread@@QAE@I@Z 10005a15 f   IlmThreadPool.obj
 0001:00004a1f       __unwindfunclet$?setNumThreads@ThreadPool@IlmThread@@QAEXH@Z$0 10005a1f f   IlmThreadPool.obj
 0001:00004a27       __unwindfunclet$?setNumThreads@ThreadPool@IlmThread@@QAEXH@Z$1 10005a27 f   IlmThreadPool.obj
 0001:00004a32       __unwindfunclet$?setNumThreads@ThreadPool@IlmThread@@QAEXH@Z$2 10005a32 f   IlmThreadPool.obj
 0001:00004a3d       __ehhandler$?setNumThreads@ThreadPool@IlmThread@@QAEXH@Z 10005a3d f   IlmThreadPool.obj
 0001:00004a47       __unwindfunclet$?addTask@ThreadPool@IlmThread@@QAEXPAVTask@2@@Z$0 10005a47 f   IlmThreadPool.obj
 0001:00004a4f       __unwindfunclet$?addTask@ThreadPool@IlmThread@@QAEXPAVTask@2@@Z$1 10005a4f f   IlmThreadPool.obj
 0001:00004a57       __ehhandler$?addTask@ThreadPool@IlmThread@@QAEXPAVTask@2@@Z 10005a57 f   IlmThreadPool.obj
 0001:00004a70       __ehhandler$?_Buynode@?$list@PAVTask@IlmThread@@V?$allocator@PAVTask@IlmThread@@@std@@@std@@IAEPAU_Node@?$_List_nod@PAVTask@IlmThread@@V?$allocator@PAVTask@IlmThread@@@std@@@2@XZ 10005a70 f   IlmThreadPool.obj
 0001:00004a80       __ehhandler$?_Buynode@?$list@PAVWorkerThread@?A0x6db1a767@IlmThread@@V?$allocator@PAVWorkerThread@?A0x6db1a767@IlmThread@@@std@@@std@@IAEPAU_Node@?$_List_nod@PAVWorkerThread@?A0x6db1a767@IlmThread@@V?$allocator@PAVWorkerThread@?A0x6db1a767@IlmThread@@@std@@@2@XZ 10005a80 f   IlmThreadPool.obj
 0001:00004a90       __ehhandler$?_Buynode@?$list@PAVTask@IlmThread@@V?$allocator@PAVTask@IlmThread@@@std@@@std@@IAEPAU_Node@?$_List_nod@PAVTask@IlmThread@@V?$allocator@PAVTask@IlmThread@@@std@@@2@PAU342@0ABQAVTask@IlmThread@@@Z 10005a90 f   IlmThreadPool.obj
 0001:00004aa0       __unwindfunclet$?_Incsize@?$list@PAVTask@IlmThread@@V?$allocator@PAVTask@IlmThread@@@std@@@std@@IAEXI@Z$0 10005aa0 f   IlmThreadPool.obj
 0001:00004ab2       __unwindfunclet$?_Incsize@?$list@PAVTask@IlmThread@@V?$allocator@PAVTask@IlmThread@@@std@@@std@@IAEXI@Z$2 10005ab2 f   IlmThreadPool.obj
 0001:00004ac4       __ehhandler$?_Incsize@?$list@PAVTask@IlmThread@@V?$allocator@PAVTask@IlmThread@@@std@@@std@@IAEXI@Z 10005ac4 f   IlmThreadPool.obj
 0001:00004ad0       __unwindfunclet$??0logic_error@std@@QAE@ABV01@@Z$0 10005ad0 f   IlmThreadPool.obj
 0001:00004ae2       __ehhandler$??0logic_error@std@@QAE@ABV01@@Z 10005ae2 f   IlmThreadPool.obj
 0001:00004af0       __ehhandler$?_Buynode@?$list@PAVWorkerThread@?A0x6db1a767@IlmThread@@V?$allocator@PAVWorkerThread@?A0x6db1a767@IlmThread@@@std@@@std@@IAEPAU_Node@?$_List_nod@PAVWorkerThread@?A0x6db1a767@IlmThread@@V?$allocator@PAVWorkerThread@?A0x6db1a767@IlmThread@@@std@@@2@PAU342@0ABQAVWorkerThread@?A0x6db1a767@IlmThread@@@Z 10005af0 f   IlmThreadPool.obj
 0001:00004b00       __unwindfunclet$?_Incsize@?$list@PAVWorkerThread@?A0x6db1a767@IlmThread@@V?$allocator@PAVWorkerThread@?A0x6db1a767@IlmThread@@@std@@@std@@IAEXI@Z$0 10005b00 f   IlmThreadPool.obj
 0001:00004b12       __unwindfunclet$?_Incsize@?$list@PAVWorkerThread@?A0x6db1a767@IlmThread@@V?$allocator@PAVWorkerThread@?A0x6db1a767@IlmThread@@@std@@@std@@IAEXI@Z$2 10005b12 f   IlmThreadPool.obj
 0001:00004b24       __ehhandler$?_Incsize@?$list@PAVWorkerThread@?A0x6db1a767@IlmThread@@V?$allocator@PAVWorkerThread@?A0x6db1a767@IlmThread@@@std@@@std@@IAEXI@Z 10005b24 f   IlmThreadPool.obj
 0001:00004b30       __unwindfunclet$??0length_error@std@@QAE@ABV01@@Z$1 10005b30 f   IlmThreadPool.obj
 0001:00004b42       __ehhandler$??0length_error@std@@QAE@ABV01@@Z 10005b42 f   IlmThreadPool.obj
 0001:00004b50       __unwindfunclet$?errorString@?A0x80da50f8@IlmThread@@YA?AV?$basic_string@DU?$char_traits@D@std@@V?$allocator@D@2@@std@@XZ$0 10005b50 f   IlmThreadSemaphoreWin32.obj
 0001:00004b6a       __ehhandler$?errorString@?A0x80da50f8@IlmThread@@YA?AV?$basic_string@DU?$char_traits@D@std@@V?$allocator@D@2@@std@@XZ 10005b6a f   IlmThreadSemaphoreWin32.obj
 0001:00004b74       __unwindfunclet$??0Semaphore@IlmThread@@QAE@I@Z$0 10005b74 f   IlmThreadSemaphoreWin32.obj
 0001:00004b80       __unwindfunclet$??0Semaphore@IlmThread@@QAE@I@Z$1 10005b80 f   IlmThreadSemaphoreWin32.obj
 0001:00004b8c       __ehhandler$??0Semaphore@IlmThread@@QAE@I@Z 10005b8c f   IlmThreadSemaphoreWin32.obj
 0001:00004b96       __unwindfunclet$?wait@Semaphore@IlmThread@@QAEXXZ$0 10005b96 f   IlmThreadSemaphoreWin32.obj
 0001:00004ba2       __unwindfunclet$?wait@Semaphore@IlmThread@@QAEXXZ$1 10005ba2 f   IlmThreadSemaphoreWin32.obj
 0001:00004bae       __ehhandler$?wait@Semaphore@IlmThread@@QAEXXZ 10005bae f   IlmThreadSemaphoreWin32.obj
 0001:00004bb8       __unwindfunclet$?post@Semaphore@IlmThread@@QAEXXZ$0 10005bb8 f   IlmThreadSemaphoreWin32.obj
 0001:00004bc4       __unwindfunclet$?post@Semaphore@IlmThread@@QAEXXZ$1 10005bc4 f   IlmThreadSemaphoreWin32.obj
 0001:00004bd0       __ehhandler$?post@Semaphore@IlmThread@@QAEXXZ 10005bd0 f   IlmThreadSemaphoreWin32.obj
 0001:00004bda       __unwindfunclet$?value@Semaphore@IlmThread@@QBEHXZ$0 10005bda f   IlmThreadSemaphoreWin32.obj
 0001:00004be6       __unwindfunclet$?value@Semaphore@IlmThread@@QBEHXZ$1 10005be6 f   IlmThreadSemaphoreWin32.obj
 0001:00004bf2       __ehhandler$?value@Semaphore@IlmThread@@QBEHXZ 10005bf2 f   IlmThreadSemaphoreWin32.obj
 0001:00004c00       __unwindfunclet$??0sentry@?$basic_ostream@DU?$char_traits@D@std@@@std@@QAE@AAV12@@Z$0 10005c00 f   IlmThreadSemaphoreWin32.obj
 0001:00004c08       __ehhandler$??0sentry@?$basic_ostream@DU?$char_traits@D@std@@@std@@QAE@AAV12@@Z 10005c08 f   IlmThreadSemaphoreWin32.obj
 0001:00004c20       __unwindfunclet$??1sentry@?$basic_ostream@DU?$char_traits@D@std@@@std@@QAE@XZ$0 10005c20 f   IlmThreadSemaphoreWin32.obj
 0001:00004c28       __ehhandler$??1sentry@?$basic_ostream@DU?$char_traits@D@std@@@std@@QAE@XZ 10005c28 f   IlmThreadSemaphoreWin32.obj
 0001:00004c40       __unwindfunclet$??$?6U?$char_traits@D@std@@@std@@YAAAV?$basic_ostream@DU?$char_traits@D@std@@@0@AAV10@PBD@Z$2 10005c40 f   IlmThreadSemaphoreWin32.obj
 0001:00004c48       __unwindfunclet$??$?6U?$char_traits@D@std@@@std@@YAAAV?$basic_ostream@DU?$char_traits@D@std@@@0@AAV10@PBD@Z$3 10005c48 f   IlmThreadSemaphoreWin32.obj
 0001:00004c50       __ehhandler$??$?6U?$char_traits@D@std@@@std@@YAAAV?$basic_ostream@DU?$char_traits@D@std@@@0@AAV10@PBD@Z 10005c50 f   IlmThreadSemaphoreWin32.obj
 0001:00004c60       __unwindfunclet$?start@Thread@IlmThread@@QAEXXZ$0 10005c60 f   IlmThreadWin32.obj
 0001:00004c69       __ehhandler$?start@Thread@IlmThread@@QAEXXZ 10005c69 f   IlmThreadWin32.obj
 0001:00004c80       ??__EgThreadPool@IlmThread@@YAXXZ 10005c80 f   IlmThreadPool.obj
 0001:00004cb0       ??__FgThreadPool@IlmThread@@YAXXZ 10005cb0 f   IlmThreadPool.obj
